:1000000029C0000042C0000040C000003EC0000007
:1000100084C000003AC0000038C0000036C00000B4
:1000200052C0000032C0000030C000002EC00000EE
:100030002CC000002AC0000028C0000026C000001C
:1000400024C0000022C0000020C000001EC000002C
:100050001CC0000011241FBECFE5D4E0DEBFCDBF21
:1000600010E0A0E6B0E0E0EEF6E002C005900D92F0
:10007000AC38B107D9F710E0ACE8B0E001C01D9290
:10008000A53CB107E1F705D129C3BACF10928C0086
:100090008CB59DB59093C0008093BF008091B8004F
:1000A0009091B900A091BA00B091BB008093C100BB
:1000B0009093C200A093C300B093C40080918C00C1
:1000C000882321F708951F920F920FB60F921124E3
:1000D0008F939F93AF93BF938091B8009091B90095
:1000E000A091BA00B091BB000196A11DB11D8093F3
:1000F000B8009093B900A093BA00B093BB00809170
:100100008C008F5F80938C00BF91AF919F918F91F6
:100110000F900FBE0F901F9018951F920F920FB661
:100120000F9211248F938091B7008BBB15BC8F91D8
:100130000F900FBE0F901F9018955D9BFECF8CB94E
:1001400008950F931F93CF93DF93062FEC0110E0D8
:1001500003C08991F2DF1F5F1017D8F3DF91CF91B1
:100160001F910F910895CF93DF93E7DFCFEBD0E09E
:100170008D81E3DF219780E0C93BD807C9F7DF9184
:10018000CF910895FC012091BD003091BE00809177
:10019000BF009091C000280F391F318320838091C8
:1001A0008D0090918E00AC0160E070E08091C10004
:1001B0009091C200A091C300B091C400480F591F94
:1001C0006A1F7B1F42835383648375838091BF00C2
:1001D0009091C0002817390740F44F5F5F4F6F4F71
:1001E0007F4F4283538364837583089510928C00FC
:1001F0005F9904C080918C008230D0F380918C0094
:1002000008958FE890E060EE70E046E050E036D26E
:10021000809190008F3FB1F488EF80938F0082E04F
:10022000809390001092910084EB80939200109242
:100230009300109294008FE890E060EE70E046E04A
:1002400050E02CD280918F008093BC001092B700B8
:100250008091900080FF03C080EF8093B700809171
:10026000B7008BBB9091920080E020919100820FAB
:10027000911D9093BE008093BD009091940080E00A
:1002800020919300820F911D90938E0080938D009A
:10029000089584B7806884BF84B7806884BF80B7BE
:1002A000846080BF80EF8ABB13E017BB18BAA9DF58
:1002B00010BC19B988E18AB982E08EBD15BC78946A
:1002C00089B7846489BFBB24AA24A39499245F9B23
:1002D00019C12CB1293521F4D9DE89E544DFF7CFE6
:1002E000203158F530E0A90142705070E5E0440F2C
:1002F000551FEA95E1F7C9018470907073E0880F8B
:10030000991F7A95E1F7482BC9019695982F882770
:1003100097958795482B28703070220F331F422BFA
:100320008091B700811140954BBB8091BC008F3FFD
:1003300071F284BD87E085BDCACF2F3321F48FE3EE
:10034000FCDE8B2D16C0283551F480E690E065E187
:10035000F8DEC098C198AA2499249394B8CF28377E
:1003600019F4C09AC19AB0CF253429F485E4E5DEAA
:100370008A2DE3DEACCF992021F4223411F4E6C5B6
:10038000A6CF273409F069C01ABA27B986E886B91A
:1003900089B78F7B89BF82E085BD86E790E068E002
:1003A000D0DEC0E0D1E05F9BFECF8CB1823031F572
:1003B0008FEF84BD8E01EE24FF241CC084B58823FA
:1003C000E9F7369A3699FECF84B1B7DE85B190E071
:1003D0000F2C02C0880F991F0A94E2F7E82A82E0E6
:1003E000F80E98E0F91621F48E2DA7DEEE24FF24F6
:1003F000015010400115110509F7D5CF8E3671F463
:10040000F5DE823018F48CB1D82FC0E0EFDE8230F8
:1004100050F68CB190E0C82BD92BC5CF833439F47A
:10042000E5DE823008F0BFCF8CB187B9BCCF86340F
:1004300039F4DCDE823008F0B6CF8CB185BDB3CFA5
:10044000823519F08FE379DEAECF16B889B78064B4
:1004500089BF15BC80EF8ABB3ACF253699F4C6DE3A
:10046000823008F034CFACB085E667DE8A2DA2FE7C
:1004700002C0C09A01C0C09883FF02C0C19A27CFB2
:10048000C19825CF203129F5B1DE823008F01FCF89
:10049000FCB0ACDE823008F01ACF0CB110E00AC01C
:1004A000A5DE823030F48CB1E12FF0E0E157FF4F50
:1004B00080831F5F1017A0F38FE890E06F2D70E02E
:1004C000402F50E0EBD0EFEDEF1508F000CF99DEB4
:1004D000FECE213109F0FBCE89DE823008F0F7CE66
:1004E0000CB184DE823008F0F2CE1CB18FE890E0CF
:1004F000602F70E0412F50E0C1D08FE890E0612F75
:1005000020DEE5CE80B39CE0D92ED822DD0CDD0CB8
:1005100082958F70D82A86B382958074D82ADB148E
:1005200009F4D5CEB3DDC4E0D0E041E050E00C2EBC
:1005300002C0440F551F0A94E2F7642F742F7D21E7
:10054000272F30E08B2D90E084239523281739073F
:1005500069F1772349F1B42A8E01025010408A2DA7
:1005600090E0002E02C0959587950A94E2F780FFEF
:100570001DC0992031F0FE01EC57FF4F8081F3DD63
:1005800002C0842FDADD81E090E002C0880F991F5D
:100590000A95E2F78095A822C43011F4C09806C0ED
:1005A000C53021F4C19802C06095B6222196C730AB
:1005B000D10509F0BACF8FE9E82E80E0F82E00E0EF
:1005C00010E02091C1003091C2004091C3005091D1
:1005D000C400602FF70182819381A481B58128171F
:1005E00039074A075B0708F43EC0281739074A074E
:1005F0005B0749F42091BF003091C0008081918158
:100600002817390780F1C1E0D0E002C0CC0FDD1F10
:100610006A95E2F74C2F5C2F5D21252F30E08B2D62
:1006200090E08C239D2328173907E9F0552359F0D2
:10063000BC2AC701A7DDA0FE16C0992091F0F801E1
:10064000EC57FF4F0BC04095B422C7019BDDA1FEC4
:100650000AC0992031F0F801E158FF4F808183DD15
:1006600002C08C2F6ADD0F5F1F4F86E090E0E80E1E
:10067000F91E0430110509F0A4CF29CEDC01CB010D
:10068000FC01E199FECF06C0FFBBEEBBE09A3196BC
:100690000DB20D9241505040B8F70895DC01A40FFF
:1006A000B51F4150504040F0CB01840F951F2E9153
:1006B00005D041505040D8F70895262FE199FECF3C
:1006C0009FBB8EBBE09A01970DB2021631F02DBB95
:1006D0000FB6F894E29AE19A0FBE0895F894FFCF0E
:1006E000555354435254424F582C393231363030DE
:1006F0002C76342E37005254426F784144430032F6
:0C070000343638003133353761303900B1
:00000001FF
